:020000040000FA
:0400000066303A2804
:040004000034003490
:08000800A000030EA100831209
:100010008B1C32288B1032181428B21C3228643002
:10002000010203183128182800001628172818285C
:1000300019281A281B281C281D281E281F283210A2
:10004000B214A810031005190314AA0DA90DA80DC8
:10005000B10B322832152A08AF002908AE00280853
:10006000AD00B21081010B11210E8300A00E200EF5
:02007000090085
:0C007400203084008001840A80300402E7
:10008000031C3C281230B100632183160C30850517
:1000900087018312850187010730990000309A009B
:1000A000103083168E008312603083168F00831207
:1000B0000030831691009F008312C83083168100A0
:1000C000831231309000003083168C008312103080
:1000D0008B00BD1B7128851971286400851D6D2852
:1000E000B021AD2181018E018F010B118B100B10FE
:1000F0008C018B178A203219A0204521B40B882847
:10010000031085190314BA0DF0303A020319F120D7
:10011000DF217A286400321808000B1D08000B113B
:10012000B21032141230B100051D9B28331483160F
:10013000011383120800331083160117831208007D
:1001400032110130B7008B132030370783169B0024
:100150001C141A088312A400A500C030A506103094
:10016000370783169B001C141A088312A300003063
:10017000370783169B001C141A088312A2008B17E2
:10018000331CC82822090339A200A309A409A50920
:1001900022082D02031DEB2823082E02031DEB2845
:1001A00024082F02031DDD2801303702031DDD283E
:1001B0003E18DD283E143F147D2125082F02031D23
:1001C000EB2801303702031DEA283E1CEA283E10C6
:1001D0003F148E21EB28B70A0230370203180800BB
:1001E000A3280130B600B400B500B700850187012F
:1001F000B213A3218A20B40B0E290310851903140E
:10020000BA0DF0303A0203193529B51F8501B51F23
:100210008701B50B0E299630B5004021321DFA2812
:100220003211331C18292D090339AD00AE09AF096D
:100230002F1CB2132F1CFA28B21BFA282E18FA28EA
:10024000B2178B1320303707BC002F08BB004E219C
:1002500010303707BC002E08BB004E210030370796
:10026000BC002D08BB004E218B1785018701AA21F8
:10027000B70AB60102303702031CFA28AD21080084
:100280000130370203199A2108003F1C08003F1073
:100290001030BC003E08BB004E2108008B133B0809
:1002A00083161C159A0083123C0883169B00553058
:1002B0009D00AA309D009C1464009C185C291C11B0
:1002C00083128B170800831600309B001C141A0839
:1002D0008312BD00831610309B001C141A08831271
:1002E000BE001430CA00CB00CC00CD00CE00CF0041
:1002F000D000D100D200D30008000130BE00BD18EC
:100300000230BD190230C000C100C200C300C400E9
:10031000C500C600C700C800C90008000830C000FA
:10032000C100C200C300C400C500C600C700C800A9
:10033000C9000800380933398500B80039093F3948
:100340008700B900080011308500B800133087001D
:10035000B9000800B801B90108003E187D21080065
:10036000B601B401B5013D1CB829BD01BD14C429B5
:10037000BD1CBD29BD013D15C4293D1DC229BD01BE
:10038000BD15C429BD013D143D08B6006400C8294F
:10039000C929CA29CB29CC29B51B0516B51F0512B9
:1003A000B40BC629B50BC6290310B60CB608031D3D
:1003B000C6290030BC003D08BB004E21080054088F
:1003C0000E02031C05160318051255080E02031C25
:1003D00085160318851256080E02031C051403180F
:1003E000051057080E02031C8514031885105808C1
:1003F0000E02031C87140318871059080E02031CF1
:100400000715031807115A080E02031C07140318D6
:1004100007105B080E02031C8716031887125C087E
:100420000E02031C0716031807125D080E02031CB8
:100430008715031887118F08031908008F0185019C
:100440008701401C2B2AFF30D400CA0B6C2AC00144
:10045000C0140A30D400C01C382ACA0B6C2A1E30C3
:10046000CA00D40F6C2AD403C00140151430DE003A
:10047000401D5F2ADE0B6C2A3030DE00FF30D400D6
:10048000D500D600D700D800D900DA00DB00DC00A8
:10049000DD00CA0B6C2A85305F07DF00CA00883098
:1004A0003D19FF30BD19FF30D400D500D600D7006C
:1004B000D800D900DA00DB00DC00DD006C2AC01DAA
:1004C000672ACA0B6C2A0A30CA00D40B6C2AD401E2
:1004D0001930CA00C0016C2A411C762AFF30D500B1
:1004E000CB0B912AC101C1140A30D500C11C812A4D
:1004F000CB0B912A0F30CB00D50F912AD503C10128
:100500004115411D842A912AC11D8C2ACB0B912AA9
:100510000B30CB00D50B912AD5011430CB00C10193
:10052000912A421C9B2AFF30D600CC0BB62AC2016E
:10053000C2141930D600C21CA62ACC0BB62A0A3027
:10054000CC00D60FB62AD603C2014215421DA92AF5
:10055000B62AC21DB12ACC0BB62A0930CC00D60B64
:10056000B62AD6011430CC00C201B62A431CC02AD8
:10057000FF30D700CD0BDB2AC301C3140A30D700EC
:10058000C31CCB2ACD0BDB2A0F30CD00D70FDB2AC3
:10059000D703C3014315431DCE2ADB2AC31DD62A28
:1005A000CD0BDB2A0830CD00D70BDB2AD701143066
:1005B000CD00C301DB2A441CE52AFF30D800CE0B56
:1005C000002BC401C4140F30D800C41CF02ACE0B79
:1005D000002B0F30CE00D80F002BD803C4014415D8
:1005E000441DF32A002BC41DFB2ACE0B002B0D301B
:1005F000CE00D80B002BD8011430CE00C401002B44
:10060000451C0A2BFF30D900CF0B252BC501C51483
:100610001430D900C51C152BCF0B252B1B30CF0058
:10062000D90F252BD903C5014515451D182B252BA1
:10063000C51D202BCF0B252B0B30CF00D90B252B25
:10064000D9011430CF00C501252B461C2F2BFF30BC
:10065000DA00D00B4A2BC601C6140F30DA00C61CD4
:100660003A2BD00B4A2B0F30D000DA0F4A2BDA038B
:10067000C6014615461D3D2B4A2BC61D452BD00BEA
:100680004A2B0730D000DA0B4A2BDA011430D000A5
:10069000C6014A2B471C542BFF30DB00D10B6F2BBC
:1006A000C701C7140A30DB00C71C5F2BD10B6F2BAF
:1006B0000F30D100DB0F6F2BDB03C7014715471D40
:1006C000622B6F2BC71D6A2BD10B6F2B0C30D10007
:1006D000DB0B6F2BDB011430D100C7016F2B481CE3
:1006E000792BFF30DC00D20B942BC801C8140F30DB
:1006F000DC00C81C842BD20B942B0A30D200DC0FF8
:10070000942BDC03C8014815481D872B942BC81D6A
:100710008F2BD20B942B0630D200DC0B942BDC01F8
:100720001430D200C801942B491C9E2BFF30DD00F1
:10073000D30BB92BC901C9140A30DD00C91CA92B80
:10074000D30BB92B1430D300DD0FB92BDD03C90156
:100750004915491DAC2BB92BC91DB42BD30BB92B93
:100760000B30D300DD0BB92BDD011430D300C901F0
:04077000B92B080099
:084000000500030006000900A1
:02400E00CC33B1
:10420000010003000300030003000200020002009B
:1042100002000000000000000000FF00FF00FF009F
:10422000000000000000000000000000000000008E
:104230000000C000C000C000C000FF00FF00FF0081
:104240000100C300F300CF00FF00C300F300CF0064
:10425000FF00C300F300CF00FF00FF00FF00FF00DE
:10426000FF00FF00FF00FF00FF00FF00FF00FF0056
:10427000FF00FF00FF00FF00FF00FF00FF00FF0046
:10428000FF00FF00FF00FF00FF00FF00FF00FF0036
:10429000FF00FF00FF00FF00FF00FF00FF00FF0026
:1042A000FF00FF00FF00FF00FF00FF00FF00FF0016
:1042B000FF00FF00FF00FF00FF00FF00FF00FF0006
:1042C000FF00FF00FF00FF00FF00FF00FF00FF00F6
:1042D000FF00FF00FF00FF00FF00FF00FF00FF00E6
:1042E000FF00FF00FF00FF00FF00FF00FF00FF00D6
:1042F000FF00FF00FF00FF00FF00FF00FF00AA001B
:00000001FF
